:1000000009C00EC00DC00DC00BC00AC009C008C099
:1000100007C006C011241FBECFE9CDBFCBD0C7C1DA
:10002000EFCF18951F93CF93DF93EC019B011E81B7
:10003000E12FF0E04C8136952795CF01BF017AD1B1
:100040008E0F9F1F642F70E087D12617370728F483
:10005000411798F4141B1E8310C05B81151768F4B8
:10006000852F90E08E1B9F0B242F30E08217930783
:1000700014F45E8302C0410F4E83DF91CF911F9134
:1000800008950F931F93CF93DF93EC018D81382F49
:1000900081FF3AC09A8180E02F81022F10E0082B67
:1000A000192B30FF17C0988180E0B801681B790BCD
:1000B000CE01B8DF8E8190E0880F991F880F991FBD
:1000C0009801281B390B88818317E0F0382F20E036
:1000D0001D8216C0798160E0601B710BCE01A2DF2A
:1000E0008E81282F30E0220F331F220F331F200F65
:1000F000311F8981381730F0382F20E081E08D835F
:100100001E8233243A832F83DF91CF911F910F9169
:100110000895FC019581892F91FF06C016821782F0
:1001200080958170858302C0926095833324089501
:10013000FC01462F858181FF21C0638147FF0DC0EF
:10014000242F2195261710F021E002C0621B262FD4
:100150008681281788F426830FC08FEF90E0861BD6
:100160009109242F332727FD30952817390714F0DC
:100170002FEF02C0242F260F23830895908180FF44
:100180000CC08181860F981710F0892F8F5F863EF3
:1001900008F085EE818382830895262F290F2B3165
:1001A00008F42BE18181281710F0282F215020839B
:1001B00022830895AF92BF92CF92DF92EF92FF9287
:1001C0000F931F93CF93DF9320E826BD92E096BD57
:1001D00080E285BF83E087BB88E188BB93BF99BF7E
:1001E00084E284BB28B981E287B9332480E690E0B9
:1001F00060E070E042E150E0C3D0809171008F3F39
:1002000011F081BF03C081B780937100F6B278947A
:10021000E3E8AE2E70E8B72E63E2C62E50E2D52E8C
:1002200041ECE42E01C0F02E889580916200865E3C
:1002300086BFAFBC8895BFBC889580916A00865EFA
:1002400089BDCFBC8895DFBC20916D0030E08091E6
:10025000650090E0282B392B20FD19C0E19917C0CB
:10026000C0E6D0E000E010E0C80199D0988189177D
:1002700031F09DBBF894E29A7894E19A08C080E04E
:10028000C137D80721F021960F5F1F4FEDCF88951A
:1002900080E690E0F6DE889588E690E0F2DE8895CC
:1002A000E6B865B1332039F1162F1219193114F05F
:1002B00018E103C0183E0CF418EE809170008230F3
:1002C00058F490E033E0880F991F3A95E1F7805A8F
:1002D0009F4F612F2DDF0DC080917100810F87FF2F
:1002E00002C080E003C0853608F084E68093710088
:1002F00081BF210E07C0862F8C57883018F4332415
:100300003394262E889506B3802F80958F21182F41
:1003100084FF06C033241092700080E690E0F9DE7E
:1003200013FF81CF332481E08093700088E690E052
:10033000F0DE79CF5527002480FF02C0060E571F3C
:10034000660F771F6115710521F0969587950097C7
:1003500099F7952F802D0895AA1BBB1B51E107C06B
:10036000AA1FBB1FA617B70710F0A61BB70B881F45
:10037000991F5A95A9F780959095BC01CD010895D4
:10038000A82F862FE82FE199FECF1FBA05C0EEBB3C
:10039000E09AE3950DB20D924150C8F70895E199A6
:1003A000FECF1FBA8EBBE09A99278DB30895F894BB
:0203B000FFCF7D
:02000004008179
:100000001BE58080040000001BE5808004000000E8
:02001000FFFFF0
:02000004008278
:0200000069FF96
:00000001FF
